:020000040800F2
:10000000A0320020850100082D3E0008A52A000826
:10001000293E0008FD0200085955000800000000B4
:100020000000000000000000000000005142000835
:100030007B10000800000000CD3E00087943000856
:100040009F0100089F0100089F0100089F01000810
:100050009F0100089F0100089F0100089F01000800
:100060009F0100089F0100089F0100089F010008F0
:100070009F0100089F0100089F0100089F010008E0
:100080009F0100089F0100089F0100089F010008D0
:100090009F0100089F0100089F0100089F010008C0
:1000A0009F0100089F0100089F0100089F010008B0
:1000B0009F0100089F0100089F0100089F010008A0
:1000C0009F0100089F0100089F0100089F01000890
:1000D0009F0100089F0100089F0100089F01000880
:1000E0009F0100089F0100089F0100080000000018
:1000F0000000000000000000000000000000000000
:1001000000000000000000009F0100089F0100089F
:100110009F0100089F0100089F0100089F0100083F
:100120009F0100089F0100089F0100089F0100082F
:100130009F0100089F0100089F0100089F0100081F
:100140009F010008B9040008E90400089F010008A5
:10015000DFF80CD000F04CF8004800476D5800085C
:10016000A0320020EFF30980704780F309887047C0
:10017000EFF30880704780F30888704740BA7047F3
:10018000C0BA70470648804706480047FEE7FEE7CA
:10019000FEE7FEE7FEE7FEE7FEE7FEE7FEE7FEE737
:1001A000394400085101000840EA01039B0703D0CD
:1001B00009E008C9121F08C0042AFAD203E011F8A6
:1001C000013B00F8013B521EF9D27047D2B201E068
:1001D00000F8012B491EFBD270470022F6E710B54C
:1001E00013460A4604461946FFF7F0FF204610BDA5
:1001F000064C074D06E0E06840F0010394E8070074
:1002000098471034AC42F6D3FFF7A6FFA45B000872
:10021000C45B00080FB470B5049D9DF81A0008284F
:1002200002DD08208DF81A000C49049808609DF83A
:100230001A008872002407E00DF11B00015D0748D9
:100240000B300155601CC4B29DF81A00A042F3DCCB
:10025000284600F005F870BC5DF814FB782A0020F1
:1002600070B5044603254FF6D0702040B0F5806F7E
:1002700004D1012500201149086010E040F2DF7030
:10028000844203D040F20B70844204D10225002046
:100290000A49086003E00325002008490860012D91
:1002A00004D0022D03D0032D05D103E004E002F0B9
:1002B000F7FE01E000E000BF00BF70BDE8000020D5
:1002C00010B501214FF0C05003F002FE012003F0F1
:1002D000F7FD10BD00BF0748006800F4E060064964
:1002E0000843001D03490860BFF34F8F00BF00BFE4
:1002F000FEE700000CED00E00000FA0500BFFEE79D
:1003000002480068C043014908607047D0000020DF
:1003100000B50648006838B901200549086005485D
:100320000249086005F064F900BD0000D800002013
:10033000D40000202083B8ED4FF0FF300149086061
:1003400070470000D000002030B503460C46094835
:100350000268002108E0605C5040C5B2064850F8D1
:10036000250080EA1222491C9942F4D30148026018
:10037000002030BDD00000207826002000B589B0D4
:100380000121092003F0C4FD0121480603F0A0FD6E
:100390000121880603F09CFD4FF40050ADF82000C9
:1003A00003208DF8220018208DF8230008A940486A
:1003B00002F09BFA4FF48050ADF8200048208DF8F1
:1003C000230008A93A4802F090FA00208DF81A009C
:1003D00001208DF81B0000208DF81C008DF81D00F9
:1003E0008DF81E008DF81F008DF8160001208DF885
:1003F000170008208DF8180001208DF8190006203C
:10040000ADF8140005A92B4800F0B9FA0E208DF8BC
:100410000E0000208DF80F0001208DF81000002044
:10042000ADF80400ADF80600ADF80800ADF80A001C
:100430000120ADF80C008DF8110001A800F046F97C
:10044000012210211B4800F091FA41208DF8000094
:1004500001208DF8010000208DF8020001208DF8A8
:100460000300684603F0EAFC012005F023F90122AD
:100470005102104800F07AFA012291020D4800F072
:1004800075FA0122D1030B4800F070FA42208DF872
:10049000000001208DF8010000208DF802000120ED
:1004A0008DF80300684603F0C9FC002009B000BDC8
:1004B000000C01400068004000B587B0012005F045
:1004C00005F902AA0121074800F0E3FA0698009016
:1004D00002A80FC8FFF79EFE142102A8FFF77DFEB9
:1004E00007B000BD0068004010B54FF400712D4802
:1004F00000F0ACF9012820D12B492A4800F06AF914
:10050000012815D100BF022808DA284911F8301057
:1005100021B1264911F83010032900D104E002214D
:10052000224A02F8301000BF1F491E4800F042F86E
:100530004FF400711B4800F059F84FF480611948DE
:1005400000F084F901282BD11749891C154800F0C7
:1005500041F901281FD10124022C03DA134810F8B5
:10056000340000B912E00320104901F8340001EB17
:10057000C401081D002103F0D1FF1CB90C4800F094
:1005800089F802E0074800F085F800BF0649891C99
:10059000044800F00FF84FF48061024800F026F89C
:1005A00010BD0000006800400200F010F4000020C0
:1005B0000064004000220C4B994202D10023836169
:1005C00011E0C1F3130201F000730BB1C2600AE045
:1005D00001F080630BB1026105E001F000630BB133
:1005E000826000E0426070477000F030B1F5007F3B
:1005F0003AD00FDC202928D006DC01291CD00429A0
:100600001DD0082940D11DE0402921D0B1F5807FBF
:100610003AD126E0B1F5004F31D006DCB1F5806F5C
:1006200025D0B1F5006F2FD124E0B1F5803F12D075
:10063000B1F5003F28D111E0154A826025E008227B
:10064000C26022E01022C2601FE0082202611CE0AA
:100650001022026119E00822426016E01022426076
:1006600013E00422426010E0042242600DE0042204
:1006700042600AE0002282610422426005E000221A
:1006800082610422426000E000BF00BF70470000AA
:100690000101010010B504460B48844209D1012133
:1006A000480603F025FC00214FF0007003F020FC09
:1006B00008E00121880603F01BFC00214FF0806058
:1006C00003F016FC10BD00000064004010B50021CE
:1006D000837A012202FA03F13D4A126842F00102D4
:1006E0003B4B1A603A4A1C3212688A43384B1C331F
:1006F0001A60027BCAB9364A0C3212688A43344BFC
:100700000C331A604288C38842EA0343304A4032BD
:10071000847A42F834300288838842EA03432C4AC0
:100720004032847A02EBC4025360027B012A19D161
:10073000274A0C3212680A43254B0C331A60428850
:10074000038842EA0343224A4032847A42F8343032
:10075000C288838842EA03431D4A4032847A02EB0E
:10076000C4025360C27A3AB9194A121D12688A4308
:10077000174B1B1D1A6006E0154A121D12680A432A
:10078000134B1B1D1A60028932B9114A14321268C8
:100790008A430F4B14331A600289012A06D10C4A8E
:1007A000143212680A430A4B14331A60427B012A3E
:1007B00006D1074A1C3212680A43054B1C331A60E3
:1007C000034A126822F00102014B1A6010BD0000BA
:1007D0000066004010B50246002001F4700343B1EA
:1007E0009369C1F3130423400BB101202DE00020D5
:1007F0002BE001F0807343B15368C1F3130423402D
:100800000BB1012021E000201FE001F0006343B1A3
:100810009368C1F3130423400BB1012015E00020BD
:1008200013E001F0007343B1D368C1F31304234014
:100830000BB1012009E0002007E01369C1F31304A4
:1008400023400BB1012000E0002010BD70B504462C
:100850000D46002660692840002871D0B5F5807FDC
:100860005CD010DC082D35D006DC012D20D0022D07
:1008700024D0042D72D127E0102D31D0202D35D079
:10088000402D6BD138E0B5F5004F60D009DCB5F5EF
:10089000007F49D0B5F5806F4CD0B5F5006F5DD1C4
:1008A0004FE0B5F5803F2DD0B5F5003F56D12FE094
:1008B000A0682D4900F0D8FB064651E0E06803210E
:1008C00000F0D2FB06464BE0E068082100F0CCFBCC
:1008D000064645E0E068102100F0C6FB06463FE012
:1008E0002069032100F0C0FB064639E02069082199
:1008F00000F0BAFB064633E02069102100F0B4FB9B
:1009000006462DE06068082100F0AEFB064627E0B1
:100910006068102100F0A8FB064621E0A0690121D3
:1009200000F0A2FB06461BE0A069022100F09CFB40
:10093000064615E0A069042100F096FB06460FE08C
:100940000FE0A069702100F08FFB064608E06068A8
:10095000042100F089FB064602E0FFE7002600BF05
:1009600000E00026304670BD010101001AB1436964
:100970000B43436102E043698B434361704730B5E9
:10098000024600200023146824F002041460146856
:1009900044F00104146000E05B1C546804F001049E
:1009A0001CB94FF6FF74A342F6D1546804F0010459
:1009B0000CB900206CE08C79012C04D1146844F04F
:1009C0008004146003E0146824F080041460CC797F
:1009D000012C04D1146844F04004146003E014684E
:1009E00024F0400414600C7A012C04D1146844F003
:1009F0002004146003E0146824F0200414604C7A8E
:100A0000012C04D1146844F01004146003E014684D
:100A100024F0100414608C7A012C04D1146844F082
:100A20000804146003E0146824F008041460CC7A0D
:100A3000012C04D1146844F00404146003E0146829
:100A400024F0040414608C78A407CD7844EA05648B
:100A50000D7944EA05444D7944EA05540D886D1E2C
:100A60002C43D461146824F001041460002300E0D6
:100A70005B1C546804F001041CB14FF6FF74A342E0
:100A8000F6D1546804F001040CB1002000E001200C
:100A900030BD10B500F5D87303EB01131B6803F0EC
:100AA00004031372137A53B900F5D87303EB0113DF
:100AB0001B6840F2FF7404EA5353136009E000F529
:100AC000D87303EB01131B686FF0604404EAD3038F
:100AD000536000F5D87303EB01131B6803F00203A6
:100AE000537200F5D87303EB01135B6803F00F0337
:100AF000937200F5D87303EB01135B681B0AD37480
:100B000000F5D87303EB01139B68D37200F5D8731B
:100B100003EB01139B681C0A147300F5D87303EBF5
:100B200001139B681C0C547300F5D87303EB01137D
:100B30009B681B0E937300F5D87303EB0113DB68FE
:100B4000D37300F5D87303EB0113DB681C0A14742C
:100B500000F5D87303EB0113DB681C0C547400F52B
:100B6000D87303EB0113DB681B0E937421B9C368C0
:100B700043F02003C36003E0036943F020030361F3
:100B800010BD10B502460020936803F08063B3F1F6
:100B9000806F00D110E0936803F00063B3F1006F41
:100BA00001D1012008E0936803F08053B3F1805F26
:100BB00001D1022000E00420042874D002F5C073A3
:100BC00003EB00131B6803F0010402F5C07303EB91
:100BD00000131C600B7A7BB94B7A0C8843EA4453B0
:100BE00002F5C07404EB00142468234302F5C074BA
:100BF00004EB0014236010E00B7A4C6843EAC40352
:100C00004C7A234302F5C07404EB00142468234398
:100C100002F5C07404EB001423608B7A03F00F0319
:100C20008B7202F5C07303EB00135B6823F00F04B3
:100C300002F5C07303EB00135C6002F5C07303EBB5
:100C400000135B688C7A234302F5C07404EB001434
:100C500063608B7B1C064B7B44EA03440B7B44EABA
:100C60000323CC7A234302F5C07404EB0014A36081
:100C70008B7C1C064B7C44EA03440B7C44EA032334
:100C8000CC7B234302F5C07404EB0014E36002F54F
:100C9000C07303EB00131B6843F0010402F5C0733B
:100CA00003EB00131C6010BD10B50246002321B1F8
:100CB000012907D002290FD109E090681D4C00EAF4
:100CC00004030BE090681C4C00EA040306E0906803
:100CD0001A4C00EA040301E0002300BF00BF184CD7
:100CE000181BA34216D007DC83B16FF08060184454
:100CF00070B1022818D111E0B0F5007F10D0114C6E
:100D0000204448B1B0F5003F0ED10BE002230DE0C6
:100D100000230BE0002309E0002307E0012305E0A6
:100D2000012303E0012301E0002300BF00BFD8B28C
:100D300010BD0000030000040003000800000310C1
:100D4000000100080001FFF70FB430B585B00024A2
:100D5000142208A96846FFF727FA012004F0CAFC0C
:100D600020B9012005B030BC5DF814FB69460E487F
:100D7000FFF707FF0546002401E0601C84B2012054
:100D800004F0B8FC40B129460748FFF78DFF18B9B9
:100D900040F6FF708442F0DB40F6FF70844201DBD6
:100DA0000120DFE70020DDE70068004010B50020EB
:100DB00000F010F910BD70473048407820F0400036
:100DC0002E4948700846407820F0200048700846B8
:100DD000407820F0100048700846807820F00F001E
:100DE00088700846807820F0F00088700846007807
:100DF00020F0010008700846007820F00800087014
:100E00000846007820F0040008700846007820F0BA
:100E1000020008700846007820F02000087008469C
:100E2000007820F0100008700846007820F080005C
:100E300008700846007820F04000087008464078A6
:100E400020F0010048700846407820F00200487009
:100E50000846407820F00400487000204871C1F82E
:100E6000F000C1F8F400C1F8F800C1F8FC00C1F8C6
:100E7000EC004FF6FF70A1F8E600704768150020FF
:100E80000148007870470000EE000020014800781B
:100E900070470000ED00002010B50024002012492A
:100EA000087012490870124908701249087072B629
:100EB000FFF782FF00240DE000200F4908550F497D
:100EC00008552146012001F047FE204601F036FE7C
:100ED000601CC4B2012CEFDB00F09AF801F0C4FFF3
:100EE00003F0D2FD62B610BDEF000020EE0000203E
:100EF000F0000020ED000020F1000020F2000020B2
:100F00000949097842290DD1074949784F2909D162
:100F100005498978452905D10349C978522901D164
:100F2000012000E0002070478E00002010B5064828
:100F30000078002806DD04480078401E0249087049
:100F400003F0FCFC10BD0000F00000200248007817
:100F5000401C014908707047EE00002001490870EC
:100F600070470000ED00002010B5FFF724FF02F0ED
:100F7000EBFC04F06FF9FFF7E9FFFFF7D7FF10BDB7
:100F800010B503480078012801D104F053F910BDD1
:100F9000EF00002000204FF4AC7000E0401E00285D
:100FA000FCD1704710B50446012C00DB10BD44B9DC
:100FB0008021064801F06EFD1021054801F06AFD10
:100FC00000E000BF00BF00BFF0E7000000100140DC
:100FD000000C014010B50446012C00DB10BD74B9B3
:100FE0001021094801F054FD8021084801F052FD0C
:100FF000FFF7D0FF8021054801F04AFD00E000BF67
:1010000000BF00BFEAE70000000C014000100140F3
:1010100010B50020FFF7C6FF10BD000010B500247A
:101020000F480078012817D1FFF79EFF0D48006890
:10103000B0F5FA6F0AD3FFF7B9FE06E0601C84B280
:10104000B4F5487F01DBFFF745F9F7E7054800688D
:10105000401C0449086002E001200149087010BDED
:10106000EF000020E80000200246002002EA010311
:101070000BB1012000E000207047704700B5034627
:1010800004E0142004F06AFA581E83B2002BF8DC46
:1010900000BD00000120014908707047BA0000201F
:1010A00070B50446012501F0F7FCA04200D10025EF
:1010B000284670BD08B500210FE00A48084490F8A2
:1010C00000080DF801001DF8010007A2525C9042D3
:1010D00001D0002008BD481CC1B20429EDDB01206D
:1010E000F8E7000000300208485230315F415050AC
:1010F0000000000000B50548807800F00F000128CE
:1011000002D1FFF7D7FF00BD0120FCE768150020E2
:1011100000200549897801F00F01012901D1012042
:1011200000E0012070470000681500200246002002
:10113000A2F57143843B73B90B78632B01DD012069
:1011400008E04B783C2B01DD012003E08B781F2B5E
:1011500000DD012000E000BF00BF704710B5422055
:10116000074908704F204870452088705220C87089
:101170000A46042140F2A63000F002F910BD00003A
:101180008E000020012802D0022800D000BF704746
:10119000012802D0022800D000BF70472DE9F0419D
:1011A00004462079401CC6B22068477820688578BC
:1011B000032E03DC132003F0F9FF44E037B1032FC3
:1011C0001BD0802F03D0832F2ED117E000BF042E19
:1011D00005D0132003F0EAFF03F0F4FC32E0022014
:1011E000A081032D01DC012D03DA312003F0DEFFA5
:1011F00002E02846FFF7CCFF24E000BF042E05D014
:10120000132003F0D3FF03F0DDFC1BE00220A081DC
:10121000032D01DC012D03DA312003F0C7FF02E0CA
:101220002846FFF7AFFF0DE003F044FA18B1802025
:1012300003F0FAFF05E0002003F0F6FF122003F0B0
:10124000B5FF00BF00BF03F075FCBDE8F08170B5CD
:1012500004462079401CC6B22068457825F08005F8
:10126000022E03D1132003F0A1FF1FE0012D02D0B5
:10127000022D0CD100E000BF032E05D0132003F097
:1012800095FF03F09FFC10E00220A0810DE003F029
:1012900011FA18B1802003F0C7FF05E0002003F029
:1012A000C3FF122003F082FF00BF00BF03F042FC27
:1012B00070BD000070B50246002028E00D5C2B02D6
:1012C000002421E0134DB5F8E6505D4005F40045DB
:1012D00055B1104DB5F8E65041F2210686EA4505B4
:1012E0000C4EA6F8E65009E00A4DB5F8E6504FF668
:1012F000FF7606EA4505074EA6F8E6504FF6FF755D
:1013000005EA4303651CECB2082CDBDB401C904271
:10131000D4D370BD681500202DE9F04105460E4676
:1013200017464FF000081448807800F00F0001289D
:1013300005D01148807800F00F00022814D104F085
:101340007BFA72B60D4800683A4631464368284633
:101350009847804604F078FA62B6B8F1000F01D1E0
:10136000002402E0012400E0012414B90120BDE8BA
:10137000F0810020FBE70000681500202800002015
:1013800070B504460D4616462A462146304604F0FE
:101390000AFA70BD70B504462079401CC5B22068B9
:1013A000467826F08006022D03DC132003F0FEFEB3
:1013B0002FE0012E02D0032E1CD10DE0032D05D00D
:1013C000132003F0F3FE03F0FDFB04E00220A081F4
:1013D0000A20114908701BE0032D05D0132003F0EB
:1013E000E5FE03F0EFFB04E00220A0810A200B4998
:1013F00008700DE003F05EF918B1802003F014FFCF
:1014000005E0002003F010FF122003F0CFFE00BF24
:1014100000BF03F08FFB70BD44000020450000209A
:101420002DE9F05F06460F4690461B48B0F8E840AD
:1014300000252BE04FF44830B5FBF0F100FB1150D4
:1014400010B9404603F062FA17F805B04FEA0B29CD
:101450004FF0000A16E084EA090000F4004028B1C9
:1014600041F2210080EA440084B203E04FF6FF70AD
:1014700000EA44044FF6FF7000EA49090AF101004E
:1014800000F0FF0ABAF1080FE5DB6D1CB542D1D3BD
:101490002046BDE8F09F000068150020704710B599
:1014A0000346002003E01C5C0C54441CE0B2904254
:1014B000F9DB10BD10B50346002002E00C5C1C54A3
:1014C000401C9042FAD310BD1D48007820F08000E7
:1014D00080301B4908700020C1F8EC00C1F8F4000E
:1014E000C1F8F0000846407820F001004870084636
:1014F000007820F0020008700846007820F0040010
:1015000008700846007820F020000870084600782F
:1015100020F0010008700846007820F008000870EC
:101520000846407820F0100048700846807820F087
:101530000F0088700846807820F0F00088707047AF
:101540006815002070B506460C4615462246294609
:101550003046FFF7AFFF70BD2DE9F04F9BB0074657
:101560004FF00008C34600243879401C00F0FF0803
:1015700001201A90B8F1040F0FD0B8F1060F0CD06B
:10158000B8F1080F09D0B8F10A0F06D0B8F10C0F66
:1015900003D0132003F00AFE83E04FF0010BBBF1F0
:1015A000050F01DD4FF0050B012400255BE0012153
:1015B00001EB45013868405C0DF804001DF804009B
:1015C0004FEA002A601CC4B2022101EB45013868D1
:1015D000405C0DF804001DF8040040EA0A0A601C93
:1015E000C4B20020199000262DE0304800EB061010
:1015F0000088504525D1012019902C4800EB061099
:10160000407A012803D12A4951F8260080474FF03B
:1016100000090DE0254800EB0610406810F80900AD
:101620000DF80400601CC4B209F1010000F0FF09CC
:101630001E4800EB0610007A4845EBDC00201A90AB
:1016400003E0701CC6B2052ECFDB00BF03F084F9A7
:1016500010B100201A9008E0199810B901201A90D2
:1016600003E0681CC5B25D45A1DB00BFBC8101255C
:1016700005E01DF80500B9684855681CC5B2A542CB
:10168000F7DB1A9801280CD103F014F818B1802068
:1016900003F0CAFD05E0002003F0C6FD312003F091
:1016A00085FD03F047FA1BB0BDE8F08F3C5B0008F6
:1016B0008C5B0008002005E00449095C044A1154D1
:1016C000411CC8B20528F7DB70470000B759000875
:1016D000A8000020002005E00449095C044A1154D8
:1016E000411CC8B20928F7DB70470000AE5900085A
:1016F00035150020002004E0FF21034A1154411C4D
:10170000C8B20628F8DB7047AD0000207047000023
:10171000002005E00449095C044A1154411CC8B288
:101720000928F7DB70470000A55900082C15002098
:101730002DE9FC41044625792068467820688778A1
:101740000B2D03D0132003F031FD46E10EB9442FD9
:1017500003D0312003F02AFD3FE1C5480078C0F3F3
:10176000400018B1702003F021FD36E12068C078F8
:101770008DF80400206800798DF805002068407914
:101780008DF80600206880798DF807002068C07900
:101790008DF800002068007A8DF801002068407AFA
:1017A0008DF802002068807A8DF803009DF804000F
:1017B00000069DF8051000EB01409DF8061000EBB7
:1017C00001209DF807100844A949C1F8F8009DF8C8
:1017D000000000069DF8011000EB01409DF802108A
:1017E00000EB01209DF803100844A149C1F8FC005A
:1017F00008460078C0F3C000002857D10846D0F84A
:10180000FC00B0F5805F0AD80846D0F8F800401C0C
:1018100028B10846D0F8F8009649884203D0312014
:1018200003F0C4FCD9E09248D0F8F800914988420E
:1018300007D18F48807820F0F00010308C498870F4
:101840000CE08B48D0F8F8008B49884206D18848D4
:10185000807820F0F0002030854988708448007836
:1018600020F008000830824908700846007820F00F
:101870000200801C08700020C1F8EC00C1F8F000E4
:10188000C1F8F4004FF6FF70A1F8E6002020A1682F
:1018900048700420A16888700020A168C8700420E6
:1018A000A081FEF735FDFEF747FD96E07048D0F8C1
:1018B000F800724988420FD06D48D0F8F800B0F5B2
:1018C000601F09D06A48D0F8F800B0F1805F03D0FB
:1018D000312003F06BFC7AE06548D0F8F8006749E6
:1018E000884205D16248D0F8FC00B0F5D03F17D847
:1018F0005F48D0F8F800B0F5601F05D15C48D0F81B
:10190000FC00B0F5002F0BD85948D0F8F800B0F122
:10191000805F09D15648D0F8FC00B0F1806F03D940
:10192000312003F043FC52E051484078C0F380007E
:1019300018B9222003F03AFC49E04D48D0F8F800ED
:101940004E49884207D14A48807820F00F00401C59
:10195000474988701AE04648D0F8F800B0F5601F93
:1019600007D14348807820F00F00801C40498870E0
:101970000CE03F48D0F8F800B0F1805F06D13C4859
:10198000807820F00F00801C394988703848007832
:1019900020F00200801C364908700020C1F8EC00DD
:1019A000C1F8F000C1F8F4004FF6FF70A1F8E600AE
:1019B0002020A16848700420A16888700020A168D8
:1019C000C8700420A081FEF7A3FCFEF7B5FC2848F0
:1019D000007820F008002649087002F0BDFF98B397
:1019E0002348007820F0020021490870084600785A
:1019F00020F0400008700846007820F08000087051
:101A00000846407820F0010048700846807820F0B1
:101A10000F0088700846807820F0F0008870002061
:101A2000C1F8F800C1F8FC00C1F8F4004FF6FF70EF
:101A3000A1F8E6000020C1F8EC00C1F8F0008875BC
:101A400000210B48C17501760948007820F010008C
:101A5000074908700846407820F010004870084692
:101A6000407820F02000487003F064F8BDE8FC8165
:101A70006815002000F0002000D8BFFE00A000087C
:101A80002DE9F04105460E4600271548854220D134
:101A9000B6F5D03F1DD803F0CFFE72B611480068EE
:101AA00001218268104890470746012F02D100208B
:101AB000BDE8F0810B4800683321826808489047F0
:101AC000074603F0C1FE62B60FB9002402E001240C
:101AD00000E001240CB90120EAE70020E8E700005B
:101AE00000A00008280000200038020870B5044655
:101AF0004FF6FF762579012D03D0132003F056FB16
:101B000086E04548007800F0010040B14248407846
:101B1000C0F3800018B9222003F048FB78E03E486B
:101B20000078C0F3400020B13B484078C0F300107B
:101B300018B9242003F03AFB6AE03748007820F017
:101B400010001030344908700846407820F010002A
:101B500048700846007820F0200008700846007899
:101B600020F0020008700846407820F00400487019
:101B70000846407820F02000487000204871C1F8E5
:101B8000EC00C1F8FC00C1F8F8000846007800F04D
:101B9000010010B90020C1F8F4001F480078C0F31C
:101BA000C00018B11C48B0F8E6602DE01A488078F3
:101BB00000F00F00012808D117493722D1F8F400AE
:101BC0001649FFF72DFC06461EE01348807800F00A
:101BD0000F00022809D110493722D1F8F4004FF440
:101BE0006011FFF71DFC06460EE00B48807800F000
:101BF0000F00022808D108493722D1F8F4004FF02D
:101C00008051FFF70DFC0646FEF77AFB0120A0810C
:101C100002F090FF70BD00006815002000A00008D1
:101C20002DE9FC5F04464FF0000B257920684678CB
:101C30002068C0782168897800EB01201FFA80FABB
:101C4000042D06DA132003F0B1FA02F073FFBDE8A9
:101C5000FC9FBAF57F4F74D00ADCAAF54040A0F58E
:101C6000FF5068B16FF48151084400286AD121E027
:101C70006FF47F405044002877D00128F6D168E007
:101C800002F05CFE032803D07F2003F08FFA10E0FF
:101C9000052D03D0132003F089FA0AE0012E03D0AA
:101CA000122003F083FA04E00020A16808710520E7
:101CB000A08163E12068007900062168497900EB82
:101CC00001402168897900EB01202168C97900EB86
:101CD0000109082D03D0132003F068FA38E0012E23
:101CE00003D0122003F062FA32E0A7480078C0F374
:101CF000001018B9222003F059FA29E0312002F02F
:101D000005FE4846FFF7CCF9E8B99F48807800F017
:101D10000F00012802D19C49C87002E001209A49B5
:101D200008719948007820F010009749087008461B
:101D3000007820F00100401C08700020A1680871A4
:101D400004E025E00CE10120A16808710520A081D4
:101D500014E102F0F3FD032808D002F0EFFD0228A1
:101D600004D07F2003F022FA11E0B4E0042D03D068
:101D7000132003F01BFA0AE0012E03D0122003F017
:101D800015FA04E00020A16808710520A081F5E0A3
:101D90000D2D03D120680079442803D0132003F0CF
:101DA00005FA97E0012E03D0122003F0FFF991E02D
:101DB000206840798DF80400206880798DF805004E
:101DC0002068C0798DF806002068007A8DF8070039
:101DD0002068407A8DF800002068807A8DF8010034
:101DE0002068C07A8DF802002068007B8DF803001F
:101DF0009DF8040000069DF8051000EB01409DF8D9
:101E0000061000EB01209DF8071047189DF8000010
:101E100000069DF8011000EB01409DF8021000EB58
:101E200001209DF8031000EB0108584887424ED16D
:101E3000B8F5D03F05D8544880780121B1EB101F88
:101E400018D05148007820F002004F490870084629
:101E5000007820F0080008700846407820F0400024
:101E600048700846807820F0F0008870312003F038
:101E70009DF92FE0312002F049FD41463846FFF739
:101E8000FFFD01281FD14048407820F00400001DCC
:101E90003D4948700846407820F0400048700846A8
:101EA000407820F00800487000F064FA0020A16833
:101EB00008710520A0813448007820F00100401C02
:101EC0003149087006E0722003F070F902E0312019
:101ED00003F06CF952E0042D03D0132003F066F9EF
:101EE0003DE0012E03D0122003F060F937E02648D0
:101EF0004078C0F3801018B9222003F057F92EE083
:101F0000FFF7F8F801281ED1FFF702F901281AD1CE
:101F10001D480079012816D11B48C078012812D12C
:101F2000FFF71CF91848407820F0080008301649DF
:101F300048700020A16808710520A0810020124986
:101F40000871C87002E0222003F030F900200E4929
:101F5000C1F8F4000846807820F00F0088700DE08A
:101F600002F0A8FB18B1802003F05EF905E0002024
:101F700003F05AF9312003F019F900BF00BF02F055
:101F8000D9FD00BF63E600006815002000A000082E
:101F90002DE9FE43054602F0D7FC07462879401C90
:101FA000C6B2286890F80180022E03DC132003F0EB
:101FB000FDF8CDE1B8F1010F09D0B8F1020F6CD0F6
:101FC000B8F1050F6FD0B8F1060F6DD13EE1012FCA
:101FD00003D17F2003F0EAF85EE0032E03D0132044
:101FE00003F0E4F858E0DC48007801280ED1A96835
:101FF0004870002405E00021A01CAA681154601C50
:10200000C4B2042CF7DB0620A88145E0D348007A4F
:10201000012803D0D148807A012803D1372003F06A
:10202000C5F839E00120A9684870CD48007801283A
:1020300012D1CA48007B03280EDB362003F0B6F825
:102040000120C649887200208880C648007810B9EF
:102050000120C44908707AE1C148007810B9C2482B
:1020600002F0C6F8002406E0BF48015DA01CAA6883
:102070001154601CC4B2042CF6DB02ABBB4A042131
:10208000B94802F02DF80020B449087208800120F8
:10209000B34908700620A88159E1012F05D17F209E
:1020A00003F084F868E068E043E1072E03D01320D2
:1020B00003F07CF860E0AA480078012859D100209C
:1020C000A7490870A548807A012803D1362003F07B
:1020D0006DF849E0002406E0A01C2968085C0DF8B2
:1020E0000400601CC4B2042CF6DB9DF800008DF8DF
:1020F00004009DF801008DF805009DF802008DF8A0
:1021000006009DF803008DF80700042201A99748F6
:1021100001F0D4FF90B10220A9684870A881002086
:1021200003F04AF801208C49087000208D4908709E
:102130008A49087302208E49087015E0352003F0A3
:1021400035F88648007B401C844908730846007BAC
:10215000032809DB012088720020888081480078EC
:1021600010B901207F49087000207C49088008725E
:1021700002E0242003F01AF8E9E0012F03D17F20C8
:1021800003F014F861E0032E03D0132003F00EF8DF
:102190005BE07148407801280FD10520A96848709C
:1021A000002405E00021A01CAA681154601CC4B2E0
:1021B000042CF7DB0620A88147E06848407A012814
:1021C00003D06648C07A012803D1372002F0EEFF21
:1021D0003BE00520A968487061484078012812D189
:1021E0005E48407B03280EDB362002F0DFFF012132
:1021F0005A48C1720021C1805A48407810B9012064
:1022000058494870A3E05648407810B9564801F044
:10221000EFFF002406E05448015DA01CAA68115499
:10222000601CC4B2042CF6DB02AB504A04214E48B9
:1022300001F09AFF00214948417200204749488037
:102240000120474948700620A88180E0012F03D172
:102250007F2002F0ABFF6BE0072E03D0132002F0CB
:10226000A5FF65E03E48407801285ED100203C494A
:1022700048703A48C07A012803D1362002F096FF10
:102280004CE0002406E0A01C2968085C0DF804005E
:10229000601CC4B2042CF6DB9DF800008DF804002D
:1022A0009DF801008DF805009DF802008DF80600EC
:1022B0009DF803008DF80700042201A92B4801F0C6
:1022C000FDFEA0B10620A96848700220A881002068
:1022D00002F072FF01202049487000202149487017
:1022E00000211E48417304202149087016E0352062
:1022F00002F05CFF1948407B401CC1B21748417393
:10230000407B03280ADB01211448C1720021C180EF
:102310001448407810B901201249487000200F4934
:10232000488000210D48417202E0242002F03EFF67
:102330000DE002F0BFF918B1802002F075FF05E052
:10234000002002F071FF122002F030FF00BF00BF3A
:1023500002F0F0FBBDE8FE83B800002068260020F4
:10236000B50000208C000020BF000020BB00002032
:10237000BA00002010B5002404E0AA200649085540
:10238000601CC4B2042CF8DB034A042140F2A630DE
:10239000FEF7F6FF10BD00008E0000202DE9F0478B
:1023A00005460024A246A146A888801E86B2286859
:1023B0004778FD4890F8058008F1010000F0FF081B
:1023C000012E02DA132002F0F1FEB6F5806F03DD74
:1023D000712002F0EBFEFCE1F3480078C0F38000CE
:1023E00050B9F148D0F8F000B0F5406F04D8EE488D
:1023F0004078C0F3001070B1EB48407820F0100036
:10240000E94948700846407820F040004870702044
:1024100002F0CCFEDDE1E4480078C0F3801028B97A
:10242000E14800780121B1EBD01F03D1722002F006
:10243000BDFECEE1DC480078C0F3400018B924208E
:1024400002F0B4FEC5E1D8484078C0F3401028B986
:10245000012F03D0732002F0A9FEBAE1781C804559
:1024600002D10220A881B4E1B84503D0732002F064
:102470009DFEAEE1CC48007800F0010040B1CA48B2
:102480004078C0F3800018B9222002F08FFEA0E14E
:10249000C548007820F020002030C3490870084665
:1024A000407820F0200020304870084647710078BE
:1024B00000F0010000287CD0002415E0A01C296851
:1024C000085CB949D1F8F010B84A5054B648D0F871
:1024D000F000401CB449C1F8F0000846D0F8F40000
:1024E000401CC1F8F400641CB442E7D32868811C86
:1024F0003046FDF729FFAC48D0F8F400AA49D1F8DE
:10250000FC10884277D3A848D0F8F000B0F5006FEF
:102510002DD3A5494FF40062D1F8F800A349FEF786
:10252000FBFE40B9FEF7D0FF722002F03FFE02F042
:1025300001FBBDE8F0879C48D0F8F80000F500608A
:102540009949C1F8F8000846D0F8F000A0F50060FD
:10255000C1F8F000002405E004F500609349085C30
:102560000855641C9048D0F8F000A042F4D88E487A
:10257000D0F8F000F0B18C48D0F8F09005E0FF20E2
:102580008A4901F8090009F10109B9F5006FF6D38C
:1025900085494FF40062D1F8F8008449FEF7BCFE8B
:1025A00040B9FEF791FF722002F000FE02F0C2FA7D
:1025B000BFE7A5E000207C49C1F8F000084640785C
:1025C00020F0010048700846007820F004000870F0
:1025D0000846007820F0200008700846407820F077
:1025E0004000403048700846407820F0100010301D
:1025F00048707EE0FFE76C48D0F8F000B0F5006F5F
:1026000077D36948407820F00100401C6649487043
:102610000846007820F00400001D08704FF40062A6
:10262000D1F8F8006149FEF777FE38B9FEF74CFFA4
:10263000722002F0BBFD02F07DFA7AE75A4800787A
:1026400020F08000584908700846D0F8F80000F5DE
:102650000060C1F8F8000846D0F8F000A0F500606E
:10266000C1F8F000002405E004F500604F49085C63
:102670000855641C4C48D0F8F000A042F4D84A48F1
:10268000D0F8EC00401C4849C1F8EC0008468078BE
:1026900000F00F00012805D10846D0F8EC00B0F595
:1026A000607F17D84048807800F00F00022805D1DD
:1026B0003D48D0F8EC00B0F5607F0BD83A48807800
:1026C00000F00F0002280ED13748D0F8EC00B0F52A
:1026D000802F08D9FEF7F8FE722002F067FD02F0A5
:1026E00029FA26E705E03048007820F040002E491E
:1026F00008702D48007820F004002B49087066E02F
:10270000B6F5805F58DA00240FE0A01C2968085C49
:102710002549D1F8F010254A50542348D0F8F0004C
:10272000401C2149C1F8F000641CB442EDD31E499D
:10273000D1F8F0001D49FEF7BDFD2868811C304628
:10274000FDF702FE1848D0F8F400194900EB010A21
:10275000154880780121B1EB101F0BD10AEB060060
:102760001449884206D21048104AD0F8F01050465A
:10277000FEF7E8FE0C48D0F8F4000B49D1F8F01051
:1027800008440949C1F8F4000846D0F8F400D1F82B
:10279000FC10884217D30448407820F01000103015
:1027A000014948700FE000006815002068160020FD
:1027B00000F00020FFFF002000200B49C1F8F400CA
:1027C000312002F0F3FC00200749C1F8F00002209C
:1027D000A8810548007820F010000349087002F035
:1027E000A9F900BFA5E60000681500202DE9F04713
:1027F000054695F8048028684078060228688078A5
:1028000006432868C71C4FF00109B8F1030F03DC29
:10281000132002F0CBFC5CE0002447E02F4800EBE3
:1028200004100088B0423FD12C4800EB0410407ADD
:10283000072839D1294800EB0410007AC01C404514
:1028400005D0132002F0B2FC4FF0000930E0394609
:102850003046FEF76BFC012805D1312002F0A6FCC2
:102860004FF0000924E00320A8811C4800EB04106D
:10287000027A1A4800EB041041683846FEF70FFE52
:10288000164800EB041000884FF28411884208D1EA
:1028900000F028F81248407820F00200801C10490F
:1028A00048704FF0000903E0601CC4B2052CB5DB92
:1028B00000BFB9F1010F0CD101F0FCFE18B180206E
:1028C00002F0B2FC05E0002002F0AEFC312002F084
:1028D0006DFC02F02FF9BDE8F08700003C5B0008BA
:1028E000681500200146FF2070472DE9F04102469F
:1028F00000250026002000230024002791F803C0B3
:102900000CF00F0591F803C00CF0100CBCF1000F97
:1029100003D091F802C04CEA050591F800C0BCF163
:10292000000F31D0146800202BE04FF0010C0CFA9E
:1029300000F3B1F800C00CEA03069E4220D18300E8
:102940004FF00F0C0CFA03F7BC4305FA03FC4CEAFA
:10295000040491F803C0BCF1280F06D14FF0010C1C
:102960000CFA00FCC2F814C00AE091F803C0BCF1F4
:10297000480F05D14FF0010C0CFA00FCC2F810C052
:10298000401C0828D1D31460B1F800C0BCF1FF0F7F
:1029900034DD546800202EE000F1080C4FF00108EF
:1029A00008FA0CF3B1F800C00CEA03069E4221D1EC
:1029B00083004FF00F0C0CFA03F7BC4305FA03FC3D
:1029C0004CEA040491F803C0BCF1280F05D100F1D2
:1029D000080C08FA0CF8C2F8148091F803C0BCF196
:1029E000480F07D100F1080C4FF0010808FA0CF865
:1029F000C2F81080401C0828CED35460BDE8F08196
:102A0000F0B50A46002300240021002500F000460E
:102A1000B6F1004F02D11D4EF16901E01B4E716805
:102A2000C0F3034583B200F44016B6F5401F08D149
:102A300021F07061154E766826F07066134F7E6047
:102A400012E000F48016B6F5801F06D1032606FAC0
:102A500005F4A14341F0706106E0460D360103FA2A
:102A600006F6B14341F0706122B1460D360103FA1A
:102A700006F6314300F00046B6F1004F02D1034E96
:102A8000F16101E0014E7160F0BD00000000014005
:102A9000416170470161704701480068704700005C
:102AA000D000002000BFFEE7704700002DE9F04F86
:102AB00095B004468A4690461E460025402105A84A
:102AC000FDF78BFB002004900027012003904FF0BE
:102AD000000B194800EB441000680490164800EB06
:102AE00044104779FF2E00D03746402F00D94027A9
:102AF000114800EB4410D0F81C90002505E019F8AF
:102B0000050005A94855681CC5B2BD42F7D305AB01
:102B1000CDE9007451464046049A00F029F88346F6
:102B2000BBF1000F02D10120039001E000200390CF
:102B3000039815B0BDE8F08FBC59000810B50446E5
:102B4000012C06DA0020034908552146012000F037
:102B500003F810BDF3000020012803D10122034B2C
:102B60005A5402E00022014B5A547047EC000020F6
:102B70002DE9F04F87B006468B4617469846DDE9AB
:102B800010954FF0000A012E03DB012007B0BDE8CD
:102B9000F08F1F48C0F8049000201D4948721D485E
:102BA00000EB4510007908701A4800EB4510407C96
:102BB00008B1012000E0002015498872154800EB9B
:102BC0004510807C08B1012000E000201049087207
:102BD00000208DF810000297084600798DF8120049
:102BE00000208DF81100002406E018F804100DF103
:102BF00013000155601CC4B29DF81200A042F4DC21
:102C00000698009002A80FC8FEF79EF85046BDE750
:102C1000902A0020BC5900082DE9F04106460C46D8
:102C2000154600270848005D08B1012C02DB002092
:102C3000BDE8F0812B46224639463046FFF736FF85
:102C400080464046F4E70000EC00002010B54FF449
:102C500000600B49086002F001FE4FF480600849F3
:102C6000091F086002F0FAFD4FF480600449086013
:102C700002F0F4FD4FF400600149091F086010BD27
:102C8000140C014010B54FF400600949086002F0CF
:102C9000E5FD4FF480600649086002F0DFFD4FF467
:102CA00080600349091D086002F0D8FD10BD0000D6
:102CB000100C014070B505460024002618E060069F
:102CC000040E4FF480600F49086002F0C7FD0D4804
:102CD0000838006800F4006008B1601CC4B24FF40A
:102CE00080600849091D086002F0B8FD701CC6B27A
:102CF000082EE4DB15B9FFF7C5FF01E0FFF7A6FFDB
:102D0000204670BD100C014070B50446002524E03B
:102D100004F0800020B14FF400601149086004E025
:102D20004FF400600E49091D086002F097FD4FF452
:102D300080600B49086002F091FD4FF48060084903
:102D4000091D0860072D02D14000091F08606006B8
:102D5000040E02F083FD681CC5B2082DD8DB70BDDF
:102D6000100C014010B54FF400600A490860401093
:102D7000086002F073FD4FF400600649091D086009
:102D800002F06CFD4FF480600249091D086002F0FA
:102D900065FD10BD100C014010B54FF400600749EF
:102DA00008604010091F086002F058FD4FF40060F1
:102DB0000249091F086002F051FD10BD140C0140CA
:102DC00010B54FF400600E49086002F047FD4FF463
:102DD00080600B49086002F041FD0948083800682E
:102DE00000F4006008B1012400E000244FF480608A
:102DF0000349091D086002F031FD204610BD0000A6
:102E0000100C014010B504460548827A0021204686
:102E1000FFF702FF012800D110BD0020FCE70000F1
:102E20001415002070B505460C46224600212846A0
:102E3000FFF7F2FE012800D170BD0020FCE7000082
:102E400010B504460448007810B900F0E1FD01E037
:102E500000F034FC10BD00006600002010B500F04A
:102E60004DFC00F01DFE10BD10B500200449087196
:102E70000449C870FF2004490870FFF7EFFF10BD38
:102E8000600000205A000020660000203EB579480E
:102E9000006878498988084401907748C0780528F7
:102EA00006D0062834D0072876D0082875D1A1E0AE
:102EB0007048C088082817DB00207049096808702E
:102EC0006C4880796D49096848706C480068801CBE
:102ED00000906848C088ADF808006649C988891C18
:102EE00088B200F00DFD12E06248807963490968FC
:102EF000087062480068401C00905E48C088ADF8C9
:102F000008005C49C988491C88B200F0F9FCA8E0B7
:102F10005849C88800F0F4FC5648C088B0F5805F76
:102F20003CDB102055490968087054480068007857
:102F300052490968087000205049096848704D4896
:102F4000C08800164D490968887000204B490968FF
:102F5000C8704848C088000A48490968087145484F
:102F6000807946490968487144480068801D00908E
:102F70004048807A801F80B2ADF808003D48807AD2
:102F8000801F3C4988800846408920F47060488151
:102F90000020394988702CE02DE060E0102037498E
:102FA000096808703548006800783249C988C1F35B
:102FB000032108433149096808702E4880792F4958
:102FC000096848702D480068801C00902948807A64
:102FD000801E80B2ADF808002648807A801E254900
:102FE00088800846408920F470604881002022498A
:102FF000887036E000BF20202049096808701F480B
:10300000006800781B494989C1F3032108431B4923
:103010000968087019480068401C00901648C0787C
:10302000082808D11348C08812498988401A80B2FC
:10303000ADF8080005E00F48807A401E80B2ADF878
:1030400008000C488188807A401E0844094988801D
:10305000BDF80810491C88B200F052FC01E00120C4
:103060003EBD00BF064801686846884704462046C2
:10307000F6E70000141500205A0000206C00002024
:1030800084000020002005E0AA21044A126811549F
:10309000411CC8B20828F7DB704700006C00002014
:1030A00070B5FE48867A082E01D0002070BDFB481E
:1030B000C07A00F0F00038B1102804D020287DD06C
:1030C00030287CD154E200BFF548007998B1F4482B
:1030D0000079012801D10020E8E7F048C07A0228F1
:1030E00026D1EE48007B3E2822D1EC48407B802848
:1030F0001ED10020DAE7E948C07A022818D1E74853
:10310000007B3E2814D1E548407B802810D1E5485B
:10311000008828B9E448008810B9E448007938B13B
:103120000020E04908800120E14908700020BDE747
:1031300000F0E4FA0220DA4908710020DD498880B5
:10314000D648C07A00F0F00000287DD010287CD14D
:10315000D2480088C0F30A0040F2DF71884206D1ED
:103160000120CF49087100F005FB00209EE7D248FE
:10317000C078022807D0D048C078032803D0CE48B2
:10318000C078082806D10120C549087100F0F2FA7C
:1031900000208BE7082E7AD1C048C07A00F00F00DB
:1031A0004FF6FF7101EA0020C249C8800846C08876
:1031B000BA49097B0843BF49C88001E0DEE06AE202
:1031C0000846C088072869DD00204881B3480D30D3
:1031D00008600B46D988B14B1B88C3F30A00B74B74
:1031E0001A689047B34908600846807A00F00300E7
:1031F00088B102280ED10320A94908800720087150
:103200000846808820F4807000F58070888000F087
:10321000BBFA42E000BFA7480068C8B39F48407BA4
:10322000A449096808709D48807BA24909684870D4
:103230009A48C07B9F49096888709848007C9D49DE
:103240000968C870954801E035E08FE0407C9949F5
:10325000096808719148807C964909684871062080
:10326000944988800846008920F00F00401C08819E
:1032700003208B490880052008710846808820F4C7
:10328000807000F58070888000F07EFA04E00BE02A
:10329000FFE700208249087100BF0AE00120804951
:1032A000087100F067FA04E001207D49087100F020
:1032B00061FA0020FAE679480088C0F30A008049E4
:1032C00008807648C07A7B49C8800846C088401C80
:1032D000B04244DC0846C08807283ADC0846C0886B
:1032E00080B3002048816D480C3008600B46D988B7
:1032F0006A4B1B88C3F30A00704B1A6890476D49EC
:10330000086008460068F0B10846807A00F00300C3
:10331000C8B9002407E061480C30005D65490968C0
:103320000855601CC4B263488079401EC0B2A042F8
:10333000F1DA01205A4908715E4AD088614A116861
:10334000884711E005E001205549087100F012FAA4
:103350000AE001205249087100F00CFA04E0012053
:103360004F49087100F006FA00209FE601204C4901
:10337000087100F0FFF900BF00BF8DE147480088E9
:10338000C0F30A0040F2DF71884206D101204449AF
:10339000087100F0EFF9002088E641480079032821
:1033A00003D03F480079052876D13D4800790528AB
:1033B0000FD13B488088C0F3002040B942490878CB
:1033C000FFF772FB40490878FFF73AFD01E0002063
:1033D0006CE638488088C01D3649C988884237DB8A
:1033E0003448C08833498988401A401CB0420EDCFA
:1033F0002A48C07A00F00F002E49097A01F00F0127
:10340000884205D001202649087100F0B3F9ACE0EC
:1034100000240AE021480C30005D26490968254A4D
:10342000928811440855601CC4B222488179007901
:10343000401C081AC0B2A042ECDA012018490871F9
:10344000002008801B4AD0881E4A116888478CE0FB
:10345000082E0BD11148C07A00F00F001549097AE7
:1034600001F00F01884202D000F048F97DE00B48DE
:10347000017B104800680F4A928881540748407BBE
:103480000C4909680B4A9288114448700348807BB4
:1034900008490968074A19E069E00000782A002015
:1034A000600000205200002054000020480000204E
:1034B00056000020201500205A0000207C0000202B
:1034C00058000020700000206800002092881144FD
:1034D00088707348C07B73490968724A92881144A6
:1034E000C8706F48017C6F4800686E4A928810442B
:1034F00001716B48407C6B4909686A4A92881144A3
:1035000048716748817C67480068664A9288104421
:10351000817164488088C01D624988800846007AAD
:10352000401C098960F303015E4801815E48807890
:10353000B0B15D488078401E5B498870084680784D
:1035400070B905200871032008800846808820F49F
:10355000807000F58070888000F016F90020A5E5E5
:103560000F20514908800320087100209EE593E058
:103570004B480088C0F30A004C49098888420ED0A5
:1035800047480088C0F30A0040F2DF71884206D144
:1035900001204549087100F0EDF8002086E5444817
:1035A000C078022807D04248C078062803D0404897
:1035B000C07807286ED13E48007900F00100A0B91C
:1035C0003B48C078062807D03948C07807280ED174
:1035D0003748807801280AD136490878FFF764FA1D
:1035E00034490878FFF72CFC01E000205EE5304804
:1035F000C07802284CD1032E4ADB2948C07A3028F3
:1036000004D0312839D032283ED13AE02848007918
:10361000C0F38000F8B92648808820F00400001D1F
:10362000234988801E48007B234908721C48457B3B
:103630000A2D02DA0120487216E005F0800058B128
:10364000F02D05DDF92D03DC01201B4948720BE04C
:103650000E201949487207E005F109000A2190FB84
:10366000F1F0401C144948721348007A10498870E0
:10367000012008800320C87009E00F200C49088051
:1036800005E000F00DFA02E000F00AFA00BF00BF0A
:1036900000200BE500E000BF00BF002006E50000B1
:1036A000782A00202015002060000020580000200B
:1036B0005A00002068000020141500200D480079F1
:1036C000052802D007280DD107E00F2009490880FE
:1036D00003200871FF20C87005E00020054908801C
:1036E000087100E0704700BFFF200349087000BF69
:1036F000F8E70000600000206600002010B51848C0
:103700000079012809DD16480079082805D008202D
:103710001349087113490868804700201049088040
:1037200008710846808820F4807088800846808868
:1037300020F4007088800C48008920F00F000A49AE
:1037400008810020488109480078802806D108496E
:103750000878FFF7A9F9FF200449087010BD0000A0
:10376000600000207400002020150020660000206A
:103770006800002010B5FFF7C1FF10BD014A50815D
:10378000704700002015002070B538488088C0F3CD
:103790004020D8B1354DA888C0F34020002863D020
:1037A0002846808820F400702946888030490878AF
:1037B000FFF728FB0446002C56D12846808820F4C9
:1037C000007000F50070294688804DE02748808809
:1037D000C0F30020002847D0244DA888C0F3002063
:1037E000002841D023480078FF283DD1802021497E
:1037F00008702846808820F4807029468880082038
:103800001D498872002605E0AA201C4909688855D0
:10381000701CC6B21848807AB042F5DC13480079B3
:10382000072804D1322015490968087003E03020C8
:103830001249096808700020104909684870012081
:103840000E4909688870002008498870084908787E
:10385000FFF7D8FA04463CB90448808820F4007089
:1038600000F500700149888070BD000060000020F4
:103870006800002066000020141500206C00002065
:1038800010B51E480088002836D01C4C208800281F
:1038900032D020460088401E214608800846008815
:1038A00040BB08460079032806D0052807D0062823
:1038B00009D007281CD103E0FFF720FF19E000BF63
:1038C000FFF71CFF15E00D48C07810B9FFF716FF91
:1038D0000DE003200949088005200871084680880A
:1038E00020F4807000F580708880FFF74DFF00E0C5
:1038F00000BF01E0FFF748FF10BD0000600000209E
:103900000C4A12780C4B03EB42125179884202DBCD
:103910000A4A91720CE0C2B2094B9A5C094B9A5C5C
:10392000064B9A721A46927A082A01DA08229A728B
:103930007047000068000020BC59000814150020E2
:10394000505900084059000810B5FFF799FF00F0E2
:1039500067F910BD10B5034609B9012010BD16481E
:10396000C07808B10320F9E71448807A082801DDFF
:10397000022200E001221148807A801A80B2884237
:1039800003DB05200C4CE07002E006200A4CE070DE
:103990000320094C2080094803600020074CA080C8
:1039A0002046C1800448808820F00100401C024C61
:1039B000A0800020D2E700005A000020141500204B
:1039C00011484089000A401C0F49498960F30B21C6
:1039D0000D4841818188807A401E80B208440A499E
:1039E000C988884203DB08200849C87002E0072024
:1039F0000649C8700320054908800846808820F0E1
:103A00000100401C88807047141500205A000020D7
:103A100010B51F48C078052806D006280ED0072804
:103A200017D008282CD100E000BF1A4801680020F8
:103A30008847002016490880C87022E00F201449EA
:103A400008800220C8700846808820F00400888022
:103A500017E00F48807860B10D488078401E0C490F
:103A600088700846807820B90F2008800220C8702E
:103A700007E00948407A064908800320C87000E042
:103A800010BD00BFFF200549087000BFF8E7000027
:103A90005A00002078000020141500206600002045
:103AA00010B501241B48C07801280EDD1948C078E4
:103AB00009280AD009201749C870174908688047A3
:103AC000044614B900201349C87000201149088029
:103AD0000846808820F0010088800846808820F011
:103AE0000200888054B10020C8700C490872084652
:103AF000408920F470604881082088720848007866
:103B000030B908490878FEF7CFFFFF200449087054
:103B100010BD00005A000020800000201415002075
:103B2000660000206800002070B539480079C0F3B5
:103B30004000D0B1364DA888C0F34000002866D0C0
:103B40002846808820F0020029468880314908787C
:103B5000FFF758F90446002C59D12846808820F0F8
:103B60000200801C2946888051E02948007900F035
:103B7000010000284BD0264DA88800F00100002845
:103B800045D025480078FF2841D1002022490870FF
:103B90002846808820F0010029468880FFF772FAC5
:103BA000FFF774F906466EB91A490878FFF72AF943
:103BB000044664BB2846808820F00200801C294609
:103BC000888024E01248C078072807D01048C078C1
:103BD000082803D00E48C07806280ED10C48C078BB
:103BE000062803D100200D49888006E00B48818813
:103BF000807A401E081A09498880FF20064908700B
:103C00000348808820F00100401C0149888070BD75
:103C10005A000020680000206600002014150020D3
:103C200010B51648008820B3144C208808B32046ED
:103C30000088401E2146088008460088D0B9084602
:103C4000C078801E072813D2DFE800F00407120CAA
:103C50000D0E0F00FFF724FF0BE0FFF7B1FEFFF79B
:103C600063FF06E000BF00BF00BFFFF719FF00E0E1
:103C700000BF01E0FFF758FF10BD00005A00002010
:103C800008B5074840680090064900980860044954
:103C90000868FCF770FA03480068804708BD000018
:103CA00000A00008E000002008B501211C2000F061
:103CB0002FF94FF40070ADF8000010208DF80300CC
:103CC00003208DF8020069465348FEF70EFE4FF4BC
:103CD00000715148FEF7DEFE0120ADF80000102013
:103CE0008DF8030003208DF8020069464A48FEF76C
:103CF000FCFD01214848FEF7CDFE40F20240ADF840
:103D0000000010208DF8030003208DF802006946A2
:103D10004148FEF7EAFD02213F48FEF7BBFE4FF4A3
:103D200080613D48FEF7B4FEA020ADF800001020F1
:103D30008DF8030003208DF8020069463748FEF72E
:103D4000D4FD20213548FEF7A3FE80213348FEF73D
:103D5000A1FE44F22720ADF8000010208DF80300EA
:103D600003208DF8020069462D48FEF7BEFD4FF492
:103D700000712B48FEF78EFE01212948FEF788FED0
:103D800002212748FEF784FE04212548FEF780FE25
:103D90004FF480412248FEF77BFE20212048FEF7A9
:103DA00077FE4FF48070ADF8000048208DF80300D6
:103DB00069461948FEF799FD4FF40070ADF8000010
:103DC00048208DF8030069461448FEF78EFD012156
:103DD000084600F09DF801211248FEF711FE102060
:103DE000ADF8000001208DF8020010208DF80300CE
:103DF00069460B48FEF779FD10210948FEF74AFE97
:103E00004FF40050ADF8000004208DF8030069461F
:103E10000248FEF76AFD08BD00080140001001409D
:103E2000000C01400001300000BFFEE7704710B5F4
:103E30004FF4A06000F03AF810BD000070B500210A
:103E400000230F22C47804B3154C246804F4E06402
:103E5000C4F5E064210AC1F10403CA40447804FABD
:103E600003F184781440214309010E4C0678A155D2
:103E7000047804F01F050124AC4005786D11AD00F5
:103E800005F1E025C5F8004109E0047804F01F05BC
:103E90000124AC40044D0678761145F8264070BDEB
:103EA0000CED00E000E400E080E100E002490143A5
:103EB000024A1160704700000000FA050CED00E0B6
:103EC000014908627047000000000E427047000080
:103ED00029B1064AD2690243044BDA6104E0034A7D
:103EE000D2698243014BDA61704700000010024042
:103EF00029B1064A12690243044B1A6104E0034ADD
:103F000012698243014B1A617047000000100240A1
:103F100029B1064A92690243044B9A6104E0034ABC
:103F200092698243014B9A61704700000010024081
:103F30002DE9F04100210022002500230026002465
:103F400000278C46DFF86081D8F8048008F00C0167
:103F500021B1042907D0082959D109E0DFF84C81A3
:103F6000C0F8008058E0DFF84481C0F8008053E0DA
:103F7000DFF83481D8F8048008F47012DFF8288163
:103F8000D8F8048008F48035920C0D2A01D0921CD8
:103F900000E0062235B9DFF8188102FB08F8C0F806
:103FA000008033E0DFF80081D8F82C8008F48036F8
:103FB000DFF8F480D8F82C8008F00F0808F101042D
:103FC00046B9DFF8E880B8FBF4F808FB02F8C0F85F
:103FD00000801BE0DFF8D080D8F82C80C8F30318ED
:103FE00008F10107DFF8C080D8F82C80C8F3032857
:103FF00008F1020CDFF8B480B8FBF7F808FB0CF806
:10400000B8FBF4F808FB02F8C0F8008004E0DFF821
:104010009C80C0F8008000BF00BFDFF88C80D8F81B
:10402000048008F0F0010909DFF8888018F80130F1
:10403000D0F8008028FA03F8C0F80480DFF8688020
:10404000D8F8048008F4E061090ADFF8688018F8FD
:104050000130D0F8048028FA03F8C0F80880DFF8AF
:104060004880D8F8048008F46051C90ADFF8448019
:1040700018F80130D0F8048028FA03F8C0F80C8052
:10408000DFF82480D8F8048008F44041890BDFF879
:10409000288018F80130D0F80C80B8FBF3F8C0F88D
:1040A0001080BDE8F08100000010024000127A008C
:1040B00000093D00000000201000002070B50346FC
:1040C0000C460120002107E0655C5E5CB54201D032
:1040D000002003E04D1CE9B29142F5DB00BF70BD4A
:1040E00078B50C46057845B9457835B9857825B950
:1040F000C57815B900251D7078BD002107E0455C25
:10410000184E765C75400DF801504D1CE9B204293B
:10411000F5DB9DF8015005F0F0059DF8006006F014
:104120000F0645EA061515709DF801502D072D0E56
:104130009DF8026045EA161555709DF8025005F08D
:10414000F0059DF8036045EA161595709DF803503B
:1041500005F00F069DF8005066F31F15D5701C7012
:1041600000BFC9E7A05B000878B50C46057845B9E3
:10417000457835B9857825B9C57815B900251D70FC
:1041800078BD002107E0455C184E765C75400DF85F
:1041900001504D1CE9B20429F5DB9DF8005005F0F3
:1041A0000F069DF8015066F31F1515709DF801501C
:1041B0002D099DF8026006F00F0645EA06155570B8
:1041C0009DF8035005F0F0059DF8026045EA1615CC
:1041D00095709DF8035005F00F059DF8006045EAC5
:1041E0001615D5701C7000BFCAE70000A05B000860
:1041F0002DE9F0410446FCF743FE054613480078DC
:104200002844C5B2002612E0691C42F2BB025143A9
:1042100043F2390202EB4100C11700EB11610912B0
:10422000A0EB0127FDB204F8015B701CC6B2042E9E
:10423000EADB06480078401C04490870084600780C
:10424000642801D100200870BDE8F081DC00002066
:10425000704710B500F002F810BD00000CB500204A
:10426000019000904048006840F480303E4908606A
:1042700000BF3D48006800F4003000900198401CE9
:104280000190009820B94FF6FF7101988842F0D153
:104290003548006800F4003010B10120009001E0C2
:1042A00000200090009801285CD13048006840F060
:1042B00010002E4908600846006820F003000860DE
:1042C0000846006840F00200086027484068264918
:1042D00048600846406848600846406840F480608E
:1042E00048600846C06A224908401F49C86208461B
:1042F000C06A204908431C49C8620846006840F06B
:104300008060086000BF1848006800F00060002866
:10431000F9D01548406820F47C10134948600846DD
:10432000406840F4E81048600846006840F080703B
:10433000086000BF0C48006800F000700028F9D049
:104340000948406820F00300074948600846406873
:1043500040F00200486000BF0348406800F00C00D5
:104360000828F9D10CBD00000010024000200240D6
:1043700000F0FEFF140801000F480068401C0E49C1
:1043800008600E480068401C0C4908600A48006834
:104390004FF47A71B0FBF1F201FB1200012804D155
:1043A00007480068401C064908600648007810B9B4
:1043B0000120044908707047340000202C000020C0
:1043C000380000203000002030B5164800684FF457
:1043D0007A72B0FBF2F1B1F1807F01D301201DE0D0
:1043E00021F07F40401E4FF0E022506150170F2215
:1043F000002807DA13071D0E0B4B00F00F04241FD3
:104400001D5503E013071C0E084B1C5400BF002071
:104410004FF0E022906107201061002008B100BF3A
:10442000FEE730BD1400002018ED00E000E400E0DD
:1044300010B5FFF725FC10BD10B51648006840F018
:1044400001001449086008464068134908401149B2
:10445000486008460068114908400E49086008464F
:10446000006820F4802008600846406820F4FE00C0
:1044700048600846006820F0A05008604FF47F00B4
:1044800088600020C862FFF7E4FE4FF00060044936
:10449000086010BD001002400000FFF0FFFFF6FEB4
:1044A00008ED00E010B50F480078401C0D49087079
:1044B000084600780A2813DB00200870FCF7E6FCA9
:1044C00070B9FCF7F7FD58B100F00EF840B10024C8
:1044D00001E0601CC4B2012CFBDB72B6FFF7A8FF41
:1044E00010BD0000E400002038B5042240F2A631DF
:1044F000684601F015F905460DB9002038BD0024C5
:1045000007E01DF80400AA2801D10020F6E7601C8E
:10451000C4B2022CF5DB0120F0E7000002460023C4
:1045200021B90D4800681060012070470A480368EF
:104530001068984205D81068181A884209D30120DB
:10454000F3E71068C0F1FF301844884201D301201E
:10455000EBE70020E9E70000340000204F48007836
:1045600001280AD14E484089401C4D49488101200C
:10457000087000204949087000E0704748484089A9
:10458000052190FBF1F201FB120030B9444840894B
:1045900018B101204249487000E0EEE740484089E8
:1045A0000A2190FBF1F201FB120028B93C48408936
:1045B00010B101203A49887039484089142190FB94
:1045C000F1F201FB120028B93548408910B10120F1
:1045D0003349C87032484089322190FBF1F201FB27
:1045E000120028B92E48408910B101202C490871C9
:1045F0002B484089642190FBF1F201FB120028B99D
:104600002748408910B10120254948712448408934
:104610004FF4FA7190FBF1F201FB120028B9204827
:10462000408910B101201E4988711D4840894FF40E
:104630007A7190FBF1F201FB120028B91848408909
:1046400010B101201649C8711548408940F2DC516B
:1046500090FBF1F201FB120028B91148408910B11A
:1046600001200F4908720E4840894FF4FA6190FB0F
:10467000F1F201FB120028B90948408910B101206C
:10468000074948720648408941F27071884202DB4E
:1046900000200349488100BF6FE700003000002080
:1046A00004010020002002490870488048607047DB
:1046B0003C00002003484078022801D101207047C7
:1046C0000020FCE75001002010B504462046FCF70E
:1046D00065FD10BD70B53848007900F04000B8B1F4
:1046E0003548007920F0400033490871012408461C
:1046F000407900B104243148007818B124F0010455
:1047000044F0020404F0010010B1002000F05AFD52
:104710002948007902281AD104202749087128481D
:104720008068007827494870002024490870244890
:104730008089C82802DA2248858900E0C825EAB2C3
:104740001F4B19699868FCF7AAFE00F049FA1A484D
:10475000007900F0100068B300201B49088017485A
:10476000007878280AD11948007838B113480078C1
:10477000782814D115484088012810D120200E49EE
:1047800008710E48007808B9012000E002200C49A9
:1047900088700F490A480161083000F0ADFE0748F3
:1047A0000078782806D109480078012802D1022033
:1047B0000149087170BD0000480000205000002031
:1047C0005001002068010020520000203C00002021
:1047D000350B002010B504462046FCF738FD10BD0F
:1047E00070B5044601252289D4E9000100F003F8E0
:1047F0000025284670BD03E0531E9AB28B5C83549B
:10480000002AF9D1704700002DE9F04104463848EC
:10481000007800F07F072068457825F0800594F83F
:104820000480B8F1010F03D1132000F0BFFC5BE05E
:10483000012D04D0022D04D0032D44D100E000BF8F
:1048400000BFB8F1020F05D0132000F0AFFC00F05C
:10485000B9F948E0012F01D1022D03D0022F07D171
:10486000032D05D17E2000F0A1FC00F0ABF93AE069
:10487000032F04D1022D02D101201D49087100200F
:1048800000F0A0FC002606E000201A4988551A49CD
:104890008855701CC6B2022EF6DBFCF7FBFB062027
:1048A000A0810020A16888703220A168C870012012
:1048B000A1680871F420A1684871032D02D101207C
:1048C000FCF74CFB0FE0FFF7F5FE20B180200B4911
:1048D0000968C87006E0002008490968C8701220FD
:1048E00000F064FC00BF00BF00F024F9BDE8F081D7
:1048F00050010020B5000020B80000204800002032
:1049000010B504462046FCF745FD10BD10B5044621
:104910000320094908707F20487008468470782079
:10492000C870AA20087148718871C87108210020D8
:10493000FEF778FA10BD0000100100200148007851
:1049400070470000500100200248007800F07F000E
:1049500070470000500100200148007870470000B7
:10496000500000200A4A127902F0FE02084B1A7128
:1049700049B91A461268824205D11A46127942F0A4
:1049800002021A7170470122024B1A7000BFF9E748
:10499000480000205600002070B504460D46A0785F
:1049A000012804D0022803D0032806D104E000BF68
:1049B000284600F057F801E000E000BF00BF0020EB
:1049C000A07070BD01460120044A127942F0010234
:1049D000024B1A711A4611600020704748000020EF
:1049E0002DE9F04104460D46002740F6C4108542EB
:1049F00003DD0220FEF7C2FE16E040F2DF708442C3
:104A000003D102200A49487006E040F20B7084424C
:104A100002D101200649487005488581FFF7D2FF81
:104A200006460EB9024887683846BDE8F0810000A6
:104A30005001002010B5044600210448FFF792FF02
:104A4000FEF798FE05200249088010BD50010020A5
:104A50005200002010B503210148FFF783FF10BD6D
:104A6000500100200021054A11800549487140216C
:104A7000034A11710121034A11707047520000204E
:104A8000480000205600002010B500201E49887004
:104A900001200870087148710020C8701B488860A8
:104AA0001B491948016100201A49487108717F208B
:104AB0001949087078208870002018490870184932
:104AC0000870FFF7EFFD1748007820F02000154927
:104AD000087000240EE0002113480155801E015586
:104AE000001F20F8141000200F490A3921F8140083
:104AF000601CC4B2022CEEDBFCF7CCFA00200B49A0
:104B000008800B49088010BD500100207101002071
:104B1000350B0020480000206801002050000020D4
:104B200056000020B3000020722600205400002010
:104B30005200002010B517480079042822D11648E9
:104B40000269846823781548007848B17F20107086
:104B5000537012480078907003210F48818208E05A
:104B60000C480068C078802803D003F14000107022
:104B7000521C0A480078782801D0FFF793FD0820DE
:104B8000044908710348007940F010000149087198
:104B900010BD0000480000205001002050000020FF
:104BA00010B504462046FCF7D7FC10BD10B50446EE
:104BB0002046FCF7BDFD10BD10B504462046FCF7AD
:104BC00095FF10BD002002490968C87070470000B9
:104BD0004800002010B504462046FDF721F810BD1E
:104BE0002DE9F05F4FF00008F8488468067B2078D4
:104BF000F749085C00EB4000F64901EB800045787E
:104C00002078F349085C00EB4000F24901EB80009A
:104C100090F804902078EE49085C00EB4000ED49E4
:104C200001EB800090F805A0FFF78EFE074694F890
:104C300000B02078862800DBC346E7480078C0F340
:104C4000401058B1E1484078022807D18020E3495C
:104C50000968C870FFF76EFFBDE8F09FDC4810F8E8
:104C60000B00FF2874D0012F04D0022F71D0032F26
:104C700070D14DE0D5484078022848D120782728C7
:104C80000ED020782E280BD020782F2808D020781E
:104C9000312805D02078342802D02078372809D14F
:104CA0007F20CF4908708020CC490968C870FFF781
:104CB00041FFD1E7607800F0800040B32078C4491C
:104CC000085C00EB4000C34901EB8000C078F0B104
:104CD0002078192802D02078282804D18020BF49C4
:104CE0000968C87013E02078B949085C00EB4000FF
:104CF000B84911F82000B04205D01320B849087017
:104D0000FFF718FFA8E78020B4490968C8709FE042
:104D1000AE48407802284BD1207827280ED0207842
:104D20002E280BD020782F2808D02078312805D0C5
:104D30002078342802D0207837280CD17F20A84949
:104D400008708020A5490968C870FFF7F3FE83E763
:104D5000C8E12EE07BE0607800F0800040B320786E
:104D60009B49085C00EB40009A4901EB8000C07849
:104D7000F0B12078192802D02078282804D180208A
:104D800096490968C87013E020789149085C00EBE7
:104D90004000904911F82000B04205D013209049FE
:104DA0000870FFF7C7FE57E780208C490968C87074
:104DB0004EE086484078022848D1207827280ED037
:104DC00020782E280BD020782F2808D02078312862
:104DD00005D02078342802D02078372809D17F20C8
:104DE0007F49087080207D490968C870FFF7A2FEDE
:104DF00032E7607800F0800040B320787449085CA6
:104E000000EB4000734901EB8000C078F0B12078DE
:104E1000192802D02078282804D180206F490968F9
:104E2000C87013E020786A49085C00EB40006949CB
:104E300011F82000B04205D0132069490870FFF72F
:104E400079FE09E7802065490968C87000E000BF65
:104E500000BF20785E49085C00EB40005D4901EB33
:104E60008000C078002875D0607800F080000028AD
:104E700071D0012E6FDD207828285AD004DC10284C
:104E800007D0112868D105E03E287CD08528F9D1CB
:104E9000D4E000BF607881280ED0607883280BD0E2
:104EA0006078822802D12078112805D06078822885
:104EB0002DD1207810282AD1022E03D01320484962
:104EC000087035E0FFF740FD012816D1062D01D00E
:104ED000042D09D1002042490870607800F080005C
:104EE0003E490968C87023E0B8F1000F20D14FF0A7
:104EF00001087E203A4908701AE0002038490870FD
:104F0000607800F0800035490968C87010E02F48CB
:104F10004078022806D1802030490968C870FFF720
:104F200009FE99E6607800F080002C490968C87095
:104F3000CDE0032E11D02548407802280DD123481A
:104F40004078022841D1802024490968C870FFF7C1
:104F5000F1FD81E6C1E0BBE0B2E06078802802D0DC
:104F60006078832823D1FFF7EFFC012815D1052DA8
:104F70000AD100201A490870607800F080001749B3
:104F80000968C87021E02DE0B8F1000F1DD14FF085
:104F900001087E201249087017E0002010490870AF
:104FA000607800F080000D490968C8700DE007487E
:104FB0004078022806D1802008490968C870FFF7A8
:104FC000B9FD49E612200649087080E05001002032
:104FD000B45A0008185A000868150020480000203C
:104FE000500000206078802819D1FFF7ADFC01281F
:104FF0000BD1042D21D1002060490870607800F0A9
:1050000080005F490968C87017E000205B4908709C
:10501000607800F080005A490968C8700DE059486E
:105020004078022806D1802055490968C870FFF7EA
:1050300081FD11E612205149087048E0022E07D088
:1050400050484078022803D113204C49087036E0BC
:105050006078812802D06078822822D1FFF774FC22
:10506000012814D1032D09D100204449087060782B
:1050700000F0800042490968C87020E0B8F1000FD4
:105080001DD14FF001087E203C49087017E0002038
:105090003A490870607800F0800039490968C870A2
:1050A0000DE038484078022806D18020344909684C
:1050B000C870FFF73FFDCFE512203049087006E0C9
:1050C000607800F080002E490968C87000BF17E0C2
:1050D00000202B490968C87012E00020284909689F
:1050E000C8700DE011202549087026484078022834
:1050F00006D1802022490968C870FFF71BFDABE587
:105100001E48007888BB022D01D1022F07D1032D44
:1051100001D1032F03D1052D07D1012F05D17F2008
:1051200016490870FFF706FD26E01648007900EAE8
:10513000090020B91348407900EA0A0028B1332059
:105140000E490870FFF7F6FC16E005200E490880AE
:1051500020780E4A105C00EB40000D4A02EB800004
:10516000816808480830884706E0FFE700200449C6
:105170000968C870FFF7DEFC00BF6DE55000002035
:10518000480000205001002052000020B45A0008BE
:10519000185A000810B504462046FCF7F9FE10BD69
:1051A0000149487170470000500100200149087012
:1051B000704700005000002001490871704700004E
:1051C0005001002070B504461248806805781148E7
:1051D0008068407800F07F06012C03D1012000F0A8
:1051E00047F904E0102D02D1304600F041F9FFF7F5
:1051F000ABFB01280CD10020FBF7B0FEFBF75AFFF8
:10520000012805D1FBF77CFE10B90A20024908707D
:1052100070BD0000500100204400002001490871C9
:10522000704700005001002001490968C8707047AC
:105230004800002010B50348007908B1FFF74AFA8A
:1052400010BD00004800002010B5FBF7E7FEFFF797
:1052500029F910BD10B500F02BF810BD70B504464B
:105260002068457825F080052679012E03D113208A
:10527000FFF79CFF19E06DB9022E05D01320FFF750
:1052800095FFFFF79FFC10E00020A1684870022006
:10529000A0810AE01220FFF789FFFFF793FCFFF7D8
:1052A00009FA10B18020FFF7BFFFFFF743FC70BD84
:1052B00010B56548008818B364480078012806D105
:1052C0000020624908704FF4FA705F490880604816
:1052D0000079A8B95C480088401E5B4908800846F0
:1052E000008868B9002008800120FFF76BFF0024C8
:1052F00004E0002057490855601CC4B2022CF8DBBA
:105300005348007900F00C00C0B153480088A8B1A0
:1053100051480088401E504908800846008868B9F6
:105320004B480068807830B9032049490968887083
:1053300000F0CEF802E0012047490880002455E043
:10534000464830F81400B0F57A7F06DB4348001D6C
:1053500030F81400B0F57A7F46DA4048001D30F886
:105360001400401C81B23D48001D20F81410001F9D
:1053700030F81400401C394921F8140001F10800EC
:10538000005D012810D1084630F81400B0F57A7F8E
:105390002ADB002021F81400002130480830015594
:1053A00000202F4908551FE02C480A30005D0128D5
:1053B0001AD12A48001D30F81400B0F57A7F13DBAB
:1053C0000020274908550021244808300155001FB6
:1053D00020F81410801D0155801C005D032803DB9C
:1053E00002211E480C300155601CC4B2022CA7DB00
:1053F0001C480078002809DD1A480078401E194929
:1054000008700846007808B9FAF764FF1648007873
:10541000002809DD14480078401E1349087008462A
:10542000007808B9FAF756FF10480078002809DD1F
:105430000E480078401E0D4908700846007808B9EB
:10544000FAF748FF10BD000054000020560000206D
:1054500048000020B80000205200002068260020EC
:10546000B500002044000020450000204600002038
:1054700010B50446FFF768FA01280AD1FFF7CEFEFF
:1054800004F07F00012810D04FF4FA700B49088017
:105490000BE004F07F00012807D1FFF7BFFE0120D9
:1054A000FFF77EFE0020054908800548047004F0DF
:1054B0007F00012801D1FBF77FFC10BD54000020C4
:1054C0005001002010B504462046FCF767FF10BDD0
:1054D00010B506490648016103218182083000F0B9
:1054E0000BF84FF4FA700349088010BD68010020E2
:1054F000500100205200002070B5044608480068A2
:10550000C078802805D0A189A068FEF723FA054657
:1055100002E00025FFF756FB284600F003F870BDB7
:105520004800002070B504460CB1032000E00020C4
:10553000054629460148FFF72FFA70BD50010020AB
:1055400010B50320FFF7EEFF002010BD10B5044694
:105550002046FDF74BF910BD00BFFEE744E03221C5
:105560003EE000BF00BF00BF00BF00BF00BF00BFE4
:1055700000BF00BF00BF00BF00BF00BF00BF00BF33
:1055800000BF00BF00BF00BF00BF00BF00BF00BF23
:1055900000BF00BF00BF00BF00BF00BF00BF00BF13
:1055A00000BF00BF00BF00BF00BF00BF00BF00BF03
:1055B00000BF00BF00BF00BF00BF00BF00BF00BFF3
:1055C00000BF00BF00BF00BF00BF00BF00BF00BFE3
:1055D00000BF00BF00BF00BF00BF00BF4A1ED1B266
:1055E0000029BEDC421ED0B20028B8DC70470000A3
:1055F000002114E0084608220BE00B4B1B68034017
:1056000023B10A4B1B6883EA500000E04008531E98
:10561000DAB2002AF1DC064B43F82100491C054BA5
:105620001B689942E6D37047D4000020D8000020C0
:1056300078260020C800002002E008C8121F08C118
:10564000002AFAD170477047002001E001C1121F03
:10565000002AFBD17047000008B501210820FEF7A1
:1056600057FC03208DF8020014208DF803004FF43E
:105670008060ADF8000069460D48FDF736F903205B
:105680008DF802004FF40060ADF8000014208DF892
:10569000030069460648FDF728F94FF48061044885
:1056A000FDF7F8F94FF400610148FDF7F3F908BD83
:1056B000000C0140022800DB70470121024A02F879
:1056C000301000BFF8E70000F4000020022803DAE1
:1056D000074911F8301001B970470121044A02F856
:1056E0003010002102EBC002517000BFF4E700004F
:1056F000F40000200146022908DA064810F83100BB
:1057000020B1044810F83100032801D1002070476F
:105710000120FCE7F400002010B5FFF79DFF10BD4D
:105720002DE9F04107460C461646FDF71BFBA0206D
:10573000FDF7EAFAFDF744FB00B130E0A046E117BF
:1057400004EB1161C1F30720FDF7DEFAFDF738FB2A
:1057500000B124E0E0B2FDF7D7FAFDF731FB00B16C
:105760001DE0FDF7FFFAA120FDF7CEFAFDF728FBBB
:1057700000B114E000250BE0711EA94201D0012107
:1057800000E000210846FDF795FA7855681C85B2BF
:10579000B542F1DBFDF700FB0120BDE8F081FDF72C
:1057A000FBFA0020F9E72DE9F04706460F46904640
:1057B0003C46002534E035B1E11704EBD1614911D5
:1057C000A4EB411109BB25B1FDF7E6FA0620FBF772
:1057D00055FCFDF7C7FAA020FDF796FAFDF7F0FAA1
:1057E00000B124E0A146E11704EB1161C1F30720E9
:1057F000FDF78AFAFDF7E4FA00B118E0E0B2FDF730
:1058000083FAFDF7DDFA00B111E0705DFDF77CFA77
:10581000FDF7D6FA00B10AE0601C84B2681C85B2BC
:105820004545C8DBFDF7B8FA0120BDE8F087FDF774
:10583000B3FA0020F9E70000014802490860704708
:1058400000F000202800002003480068006810B124
:10585000002001490860704728000020002001E076
:10586000411C88B23C28FBDB7047000086B0FEF785
:10587000E3FDFAF725FDFEF7A7FD01A8FEF758FBAB
:10588000FEF7D5FAFEF710FAFFF746FFFBF704FB29
:10589000FAF774FD4FF400712548FDF7F9F8FBF7AE
:1058A000FBFAFBF7FBFD41E0FEF758FE21480078CC
:1058B000012805D100201F49087000F03DF835E0AF
:1058C0001C484078012803D100201A4948702DE077
:1058D00018488078012805D1002016498870FFF704
:1058E000B3FC23E01348C078012803D100201149FC
:1058F000C8701BE00F480079012803D100200D4932
:10590000087113E00B484079012803D100200949B0
:1059100048710BE00748C079012807D100200549EC
:10592000C8714FF400710248FDF7B2F8BCE70000FF
:10593000000C01400401002010B5FBF721FB10BD55
:105940000001020304050607080C1014182030405B
:10595000000102030405060708090909090A0A0AE1
:105960000A0B0B0B0B0C0C0C0C0D0D0D0D0D0D0D76
:105970000D0E0E0E0E0E0E0E0E0E0E0E0E0E0E0E48
:105980000E0F0F0F0F0F0F0F0F0F0F0F0F0F0F0F28
:105990000F393231343830312D4446303200000076
:1059A000000000000056480012566E0000005648E5
:1059B0000012566E00000001170B10001B070000BC
:1059C00000080400000002000000000000000000C9
:1059D00000000000412E0008100100200B0700000D
:1059E000FF07000000000800DF070000FF070000BD
:1059F000000008002D010000FF0700000000080063
:105A00000000000000000000000000000000000096
:105A1000000000000000000002060310000000006B
:105A200009480008020603100000000001490008B0
:105A30000306030000000000A14B0008060501005A
:105A4000000000009551000803030310000000004F
:105A5000C946000814020100010000004D5500086D
:105A60000605010000000000D54B00080B020100F4
:105A700001000000AD4B0008FF0201000100000022
:105A8000C55400080102010001000000B94B0008E4
:105A900002060310000000005D520008020303101C
:105AA00000000000D54700080000000000000000D2
:105AB00000000000FFFFFFFFFFFFFFFFFFFFFFFFF2
:105AC000FFFFFFFF0001FFFFFFFFFFFFFFFFFFFFE3
:105AD000FFFFFFFFFFFF02FFFFFFFF0304FFFFFFCA
:105AE000FFFF05FFFF06FFFF07FF0809FFFFFFFF9E
:105AF000FFFF0AFFFFFFFFFFFFFFFFFFFFFFFFFFAB
:105B0000FFFFFFFFFFFFFFFFFFFFFFFFFFFFFFFFA5
:105B1000FFFFFFFFFFFFFFFFFFFFFFFFFFFFFFFF95
:105B2000FFFFFFFFFFFFFFFFFFFFFFFFFFFFFFFF85
:105B3000FFFFFFFFFFFFFFFFFF0B000094F10000DE
:105B40003515002009010000FFFF000095F100005D
:105B5000AD00002006010000FFFF000093F10000EF
:105B6000A800002005010000FFFF00008CF10000EC
:105B70003E15002013010000FFFF000080F100002F
:105B80002C15002009010000FFFF0000D5160008B9
:105B9000F5160008B51600080D17000811170008C3
:105BA0003E53E17BC45B000800000020F4000000CD
:105BB00038560008B85C0008F4000020AC31000042
:105BC000485600080000000001020304010203041B
:105BD000060708090204060800A24A0400000000A3
:105BE000000000000102030406070809000000008D
:105BF00000000000000000000000000000000000A5
:105C00000000000000000000000000000000000094
:105C10000000000000000000000000000000000084
:105C20000000000000000000000000000000000074
:105C300010010020354A0008554A00082555000883
:105C4000E149000841550008E14700080000000054
:105C50000000000000000000000000000000000044
:105C60000000000000000000000000000000000034
:105C70000000000000000000000000000000000024
:105C80000000000000000000000000000001000013
:105C900008000000000000000000000000000000FC
:105CA00000000000000000000000000000000000F4
:085CB0000000000000000000EC
:04000005080001519D
:00000001FF
